:020000040000FA
:0400040000EF08F011
:06000800010123D91100E3
:10001800D8CF00F0E0CF01F0026E010116D80250EF
:0A00280001C0E0FF00C0D8FF100087
:100040000F014FEC1CF0000102E3D8801200D890A1
:100050001200E9CF03F0EACF04F0FACF05F0FBCFAE
:1000600006F09DA813D09EA811D09D9813B105D07D
:1000700012A503D012892D8009D002EE4BF00A514F
:10008000E926EFCFADFF13810A2B00079DAA48D0C8
:100090009EAA46D0346A096AABA203D0AB98AB885B
:1000A00033D0ABA409D0AE50010E096E12A72CD0EC
:1000B0003B0EAF6E129728D03F6AAECF07F007BE57
:1000C000046B02EE0BF00451E92607C0EFFF12A704
:1000D00004D03B0EAF6E129712D013A110D002EED7
:1000E0004BF00951E926EFCF08F00750081803E05C
:1000F000010E096E04D0092B099B00679D880966D3
:1001000003D02D82042B049B13A10AD0095208E0CE
:1001100013919D9812892D80630EAF6EAD6A128780
:100120009DA687D09EA685D09E9614AB02D0149B28
:10013000416A4150E844020FF924F96E0BD016D001
:100140001DD035D03AD045D04BD050D055D05AD014
:1001500060D063D022C1C9FF212D02D0010E416EB3
:10016000020E216366D0050E416E63D0C5BC60D01F
:1001700023C1C9FF020E416E2C925BD0C5BC58D082
:100180002CB207D014B905D024C1C9FF030E416EAB
:1001900050D014A94ED02CB204D024C1C9FF2C8257
:1001A00048D025C1C9FF1499030E416E42D0C5BC89
:1001B0003FD0C584040E416E3CD0C00EC614426EC2
:1001C000426636D0216B226B236B246B416A9D966D
:1001D00030D0C5BC2DD023C1C9FF060E416E29D039
:1001E000C5BC26D0C582070E416E23D0228122C114
:1001F000C9FF080E416E1DD0C5BC1AD0C586090EB8
:10020000416E17D0C9CF24F1C58AC5880A0E416E48
:1002100010D0C5840B0E416E0CD0C00EC614426EB9
:10022000426606D0216B226B236B416A9D9601D0FA
:100230002169A1A605D0A196226B236B9D96216909
:1002400005C0FAFF06C0FBFF03C0E9FF04C0EAFFD8
:100250001200F2A80FD0F2A20DD0F292F2981285FD
:10026000346A2DB007D013B105D00D0E0F6102D046
:06027000020E0F27120030
:1004000000011EDE03E30D01F4D90001000100EF3D
:1004100008F01200146A1350146009D09E90B10EB7
:10042000CF6ECD809EA0FED7CD90142AF4D71200B7
:100430008B80126A115012600AD08B900A0E136ED4
:10044000E9DF8B80280E136EE5DF122AF3D7C80E82
:10045000136EE0DFEDD70DEE10F001010351E92638
:10046000EFCF13F00DEE10F0E926EF6A032B400EEC
:100470000361036B13500D011200152C02D0176A93
:10048000000C14C018F0182A1850166201D0186A0F
:100490000D0EEA6E18501324E96EEFCF17F01750C7
:1004A000100A03E0FD0E176EFD0C186A0D0EEA6EC1
:1004B00014501324E96EEF50181A142A14501662BF
:1004C00001D0146A1704196E19521FE0150615BEE3
:1004D00002D0156602D0176A000C0D0EEA6E145099
:1004E0001324E96EEFAE03D0FE0E176EFE0C0D0E58
:1004F000EA6E14501324E96EEF50181A142A14509F
:10050000166201D0146A1906DFD7183C02D01750C2
:1005100012001768FF0C9EAA14D0ABA203D0AB98B0
:10052000AB880FD0ABA402D0AE500BD08B900DEEA9
:1005300010F00251E926AECFEFFF022B400E026110
:10054000026B0351025D116E11AE02D0400E1126F6
:1005500011522BE00DEE10F00351E926E50EEF628B
:1005600022D0100E136E03C114F011C015F0400E0E
:10057000166E83DF17C091FD0D01915107E0FD0A52
:1005800007E0030A05E0010A06E008D001010DD0EA
:1005900062DF01010AD012680101FF0C8B80010E9D
:1005A000126E0101010C57DF0101126A000CA6B2A4
:1005B000FED711C0A9FF12C0AAFFA69EA69CA680C6
:1005C000A8501200020E1D6EA69EA69CA68418C0FE
:1005D000A9FF19C0AAFF0DEE00F01BC01CF0EFCF61
:1005E000A8FF550EA76EAA0EA76EA682A6B2FED7CA
:1005F000A680A850EF6209D0020E1D6EEE50A92A07
:10060000A950D8B4AA2A1E8002D01E9002D01C2E57
:10061000E6D71EA002D0D88012001D2EE0D7D890B9
:1006200012008B90020E256EA68EA69CA684A68E26
:1006300020C0F6FF21C0F7FF22C0F8FFA688550EA4
:10064000A76EAA0EA76EA682A6980A000DEE50F01D
:1006500023C024F0EECFF5FF0F00242EFBD7550E5C
:10066000A76EAA0EA76EA682A69420C0F6FF0DEE76
:1006700050F0268023C024F00900F550EE1802E067
:10068000269002D0242EF8D726A004D092818B8009
:10069000D8801200252ECAD7D8901200A68EA69C0C
:1006A0002250F86E2150F76EC00E2014F66E0DEE3B
:1006B00050F0400E236E0900F5CFEEFF232EFBD73E
:1006C00012003F0E18141F6E500E1F241D6E1D06C3
:1006D0001E6A1F6A1B501F5C1F501B18D8B0800A6F
:1006E00036E61D2A900E1D6219D0500E1D6E93CD58
:1006F00020F094CD21F0226A400E236E92DF0CE3AD
:10070000400E9327000E942393CD20F094CD21F03A
:10071000226AC4DF929102D0D89012000D0EEA6EC8
:100720001EC0E9FFEFCF1CF019501A1003E1030EB1
:10073000186406D00D0EEA6E1DC0E9FF1CC0EFFF65
:100740001E2A182A000E19221A221F2AC3D7D8805F
:1007500012001350176E1250166EC00E1114156E43
:100760008B80175003E1030E166407D0175005E184
:10077000010E155C0A0E16582EE317502CE1F00EF0
:10078000166029D092A10BD015C093FD16C094FD20
:1007900093CD20F094CD21F0226A80DF9291155004
:1007A00093630ED0165094630BD0176609D011C016
:1007B00018F012C019F013C01AF014C01BF081D742
:1007C00093CD20F094CD21F0226A400E236E29DFD4
:1007D000C7E2D8901200F00E136209D011C018F0D1
:1007E00012C019F013C01AF014C01BF0EBD6D88059
:1007F0001200928110928B90108001018CDEFF0A12
:100800000D0103E0FE0A07E0C6D010A2C4D0040E1A
:10081000116E0EDEC0D08B901EDE1DDE100AD8A435
:10082000BAD019DE7F0AD8A4B6D015DE7F0AD8A4C4
:10083000B2D011DE7F0AD8A4AED00DDE0A6E040E4F
:10084000010103250C6E3F0E0C6402D0400E0C5EBD
:100850000DEE10F00C50E926F00EEF140D0108E03B
:10086000100A48E0300A56E0600AD8B485D093D028
:10087000F2DD570A03E0010E116EDADDECDD180A35
:1008800003E0010E116ED4DDE6DD906F909F0AB497
:10089000908F020E010103250C6E3F0E0C6402D0F6
:1008A000400E0C5E0DEE10F00C50E926EFCF0BF071
:1008B0000D010BA00ED00BB207D09051020A09E037
:1008C000020E116EB5DD05D0020E906102D0116EE0
:1008D000AFDDC1DD906F909F0AB6908F0BA408D05A
:1008E000116A126A64DE906103D0030E116EA0DDFE
:1008F000108251D0B0DD0F6E0F9E0AB00F8EABDDAF
:100900000E6E0E9E0AB20E8EA6DD0D6E0D9E0AB400
:100910000D8E41D01DEE00F00C6A040E0C6009D063
:100920009ADDE76E0A32D8A0E69ED8B0E68E0C2A91
:10093000F4D791DD0B6E0C6A040E0C6009D08BDDD0
:10094000E76E0B32D8A0E69ED8B0E68E0C2AF4D71C
:100950000DC011F00EC012F00FC013F0080E146E8F
:10096000F8DE06E3080E0D26000E0E220F2213D02D
:10097000050E116E5DDD0FD092B10CD093CD20F03D
:1009800094CD21F0226A400E236E4BDE03E2050E69
:10099000116E4EDD109010B030D712004DBE09D050
:1009A000D6CF0AF050500A5C515E0AC050F0D8A071
:1009B0004D8E1200D6CF0AF04E500A5C4F5E0AC030
:1009C0004EF0D8B012007D0E4F26050E0B6E010EB4
:1009D0000C6E00EE43F04D500C140DE1EF06EF3CB1
:1009E00003D0EE50EF06ED50EF50EE50EF1002E165
:1009F0000C504D12ED50020EE926000EEA22D8905E
:080A00000C360B2EE8D71200A2
:101000000D0103D000EC02F00D0192B303D020ECEF
:1010100000F00D010101AEEC1CF0E1EC1CF0070149
:101020000FEC1DF04D684E6A4F6AC60ED56E2D6AE4
:10103000010152EC1DF02D862D88D08EF28EF28C9F
:10104000F28E2E6A2F6A306A316A800E406E3E6ED2
:101050003F6E366E376E3B6E3C6E3D6E346E326E5A
:10106000336E356E396E386E3A6E326A336A356A6F
:10107000376A406A396A386A3A6A0400D1900D01C9
:101080008DDC98DC2EBE02D075D82E6E2FBE04D01B
:1010900001017CD82F6E0D0130BE04D002010DD9A4
:1010A000306E0D0131BE04D0010178D9316E0D01D1
:1010B00032BE04D00101E0D9326E0D0133BE04D03E
:1010C000010171DA336E0D0134BE04D0010194D9EF
:1010D000346E0D0135BE04D00101FDD9356E0D0110
:1010E00036BE02D094DA366E37BE04D00101AADAD9
:1010F000376E0D0138BE05D00001B8EC14F0386E23
:101100000D0139BE05D001010EEC12F0396E0D0152
:101110003ABE05D00001ACEC18F03A6E0D013BBEB2
:1011200005D000014FEC17F03B6E0D013CBE05D021
:1011300000018DEC15F03C6E0D013DBE05D00001A7
:1011400015EC16F03D6E0D013EBE05D00101B4EC6C
:101150000FF03E6E0D013FBE05D00201BDEC0FF059
:101160003F6E0D0140BE8CD700011EEC19F0406EA1
:101170000D0186D7F9502E44F92601D004D0010E76
:10118000436E446A4D904DA0010C000CF9502F4461
:10119000F92601D004D00A0E456E466A4D924DA242
:1011A000010C0F6A080E0F603DD003EE00F00F50E7
:1011B000E926EFCF0CF003EE08F0E9260C50EF140F
:1011C0000E6E03EE20F00F50E9260C50EF140B6E5C
:1011D0000E500B180D6E010E0A6E0A521BE003EE44
:1011E00028F00F50E926EF500D140C6E0A500C1623
:1011F0000EE003EE20F00F50E9260A50EF1A14B16A
:1012000006D003EE40F00F50E9260A50EF12D890B6
:101210000A36E3D703EE28F00F50E9260DC0EFFFA2
:101220000F2AC0D73A6A3B6A3C6A3D6A2B0EC26EEF
:10123000C2B2FED7030EC414186FC3CF17F1180E35
:10124000175D010E185903E2A1EC11F0010113A77B
:1012500006D00201052F03D0010113978B800101F5
:1012600013A906D00201082F03D0010113998B8422
:10127000010181B008D012AF0DD00D2B0A0E0D6305
:1012800009D0129F07D00D6B12BF04D00E6702D099
:10129000010E0E6F0E530EE00E2B180E0E650AD0C7
:1012A0000E6BF29EF292F288AB889E9A9D8A9D9870
:1012B000F28E128F000C0101800CF9503044F92697
:1012C00001D004D0640E476E486A4D944DA4010CC1
:1012D00006530EE006070F0E06150AE1063B060749
:1012E0000F0E061504E0050E036F3E6A068B063BE3
:1012F000075307E0072F05D0500E036F3E6A0F0E0D
:10130000076F010112AB21D00B800A6A080E02019F
:101310000A6017D003EE40F00A50E926EF50D8A437
:101320000B9003EE60F00A50E926EF50D8A40B9022
:1013300003EE68F00A50E926EF50D8A40B900A2A71
:10134000E5D70BA002D00101129B020182B220D08E
:101350000101112B13BF08D00A0E116310D0138F97
:10136000010E0201076F0BD0020E116308D013AFFC
:1013700006D0139F0201076B650E0101116F640E09
:101380000101116303D0D19000EF00F0020102D0FF
:101390000101116B0201000C0201800CF950314473
:1013A000F92601D005D0E80E496E030E4A6E4D961F
:1013B0004DA6010C12AD1CD0128B03EE00F01051A3
:1013C000E926EFCF0AF003EE40F0E9260A50EF12CB
:1013D00003EE00F01051E926EF1C0A6E03EE40F018
:1013E0001051E9260A50EF12102B080E1061129DC1
:1013F0001491000C0101800C3444060FF924D8B07C
:10140000FA2AF96E02D007D032D01285D6CF50F02A
:10141000960E516E4D9E4DAE010CF292F2880F4524
:101420000A6EF9500A44F926960E1DD08E0E1BD076
:10143000860E19D07F0E17D0780E15D0700E13D0EF
:10144000690E11D0610E0FD05A0E0DD0520E0BD076
:101450004A0E09D0430E07D03C0E05D0340E03D0FF
:101460002D0E01D0000ED6CF50F0516E4D9E4DAED8
:10147000020C12950101800C0201F9503244F92648
:1014800000D001012DA2010C02010BAF1ED02CD9FE
:101490000A6E0A50010119E0FF0A05E102010B6B17
:1014A0000101139112D012EE0BF004EE00F0025184
:1014B000E926E6CFEEFFE950D8B404EE00F00A2E9C
:1014C000F8D7E9CF02F113912D802D922D8C0101D7
:1014D000000C0101800C3550D8A4800C0251031976
:1014E0005FE004EE00F00351E926EFAE58D004EEC1
:1014F00000F0E926EF50830A0DE0330A0FE0010AFD
:1015000021E0030A2DE05F0A39E0020A43E05B0AAA
:1015100044E045D00701D4EC0FF041D059EC0FF076
:101520000AC015F10BC016F115511615FF0A37E068
:10153000000EAAD912C00AF013C00BF092EC13F0FF
:10154000139D2DD059EC0FF00AC015F10BC016F108
:1015500015511615FF0A23E0010E96D9139D1FD0D1
:1015600059EC0FF00AC015F10BC016F11551161504
:10157000FF0A15E0020E88D9139D11D0FAEC0EF087
:101580000AC015F10BC016F115511615FF0A07E038
:10159000138D05D00AEC1AF002D007EC1CF0032BD7
:1015A000000C0101800C0201F9503344F92603D0EC
:1015B00002D017D021D001012DA4010C2D940201DD
:1015C0004B390F0B01010F6F0F0E02014B1501017B
:1015D000006F010E096F0A6F12B502D012BF03D05F
:1015E000020C0101F9D76FEC1DF012B5EDD79D8803
:1015F0002D902DB003D0030C0101FBD712A902D00E
:101600001299E2D70F6B2D86000C0101800CF95066
:101610003644F92600D02DA6010C2D9612EE2BF0A3
:10162000E6CF0AF022EE4BF00AC0DEFF0A060B6A94
:10163000E6CFDFFFDE500B1A0A2EFAD70B1CDF6E47
:101640002D84800CF9503744F92601D006D007517B
:10165000056303D00851061944E02DA6010C2D9610
:1016600022EE4BF00551E96E050E0625EA6EEFCF2E
:101670000AF00AC0DEFF052B000E0623056705D021
:10168000020E066302D0056B066B0A060B6A055153
:10169000E96E050E0625EA6EEFCFDFFFDE500B1A6E
:1016A000052B000E0623056705D0020E066302D047
:1016B000056B066B0A2EEBD70B1CDF6E0551075D21
:1016C0000A6E065108590B6E0BAE02D0020E0B26A5
:1016D0000BBE05D0D00E0A5C010E0B58D8A02D8889
:1016E0002D84000C0101800C0BAD14D00BAB0FD07E
:1016F000020E0101046101D0000C0CC20BF0030EBC
:1017000002010B6403D0100E0B640BD0FF0C060E0D
:101710000B6E07D00BAB03D0040E0B6E02D0020E83
:101720000B6E010104510B6212D00C6A0D6A02EEBD
:101730000BF00D50E926EF500C1A0D2A0B500D5CE2
:10174000F6E30C28020102E10B501200FF0C000C22
:10175000126E0F38030B136E169211BE168216947A
:1017600011B81684010116B013D016A211D012A020
:101770000FD00F0E1114186E1050176E1706000EB2
:10178000185A17C010F018C011F0119816B411882B
:101790001F0E111616B019D0135005E0010A06E00D
:1017A000030A0AE011D01186119A31D0119A1186DC
:1017B00011A82DD011962BD011341132103211985E
:1017C000D8B01188118A23D01200135005E0010A05
:1017D00009E0030A10E01AD01186100E0FBC111A8E
:1017E000119A15D0119A100E0FBC111A118611A85A
:1017F0000ED011960CD01134113210321198D8B08D
:101800001188118A080E0FBC111A01D01200D8904D
:1018100010361136D89010320751E96E050E0825A2
:10182000EA6E040EEF6EB5DB0751E96E050E082572
:10183000EA6EB00E1310EF6EACDB0751E96E050EC9
:101840000825EA6E10C0EFFFA4DB0751E96E050E14
:101850000825EA6E11C0EFFF9CDB0551075D146E91
:1018600006510859156E15AE02D0020E152615BE8A
:1018700006D0E10E145C010E1558D8B02D98050E57
:101880000201036F3E6A12000A6E0F0E1615136EE8
:101890001551126E0F6A080E0F60E8D10E68010E26
:1018A000106E1052D8B4E0D10E2A03EE00F00F50A3
:1018B000E926EF1C1014D8B4D4D10F50400DF3CF4B
:1018C000D9FFF4CFDAFF100ED926070EDA22080E60
:1018D0000E02F350D926000EDA220EA015D0080E03
:1018E000D95E000EDA5ADCCF0BF0DD501C940BBC35
:1018F0001C841C960BBE1C861CA602D01CA404D003
:10190000080ED926000EDA22DECF14F0070EDF14FF
:10191000156ED9CF1AF0DACF1BF0030ED926000EC0
:10192000DA22DECF16F0DFCF1DF00F0EDE14176EB9
:10193000DECF18F0DFCF1EF00F0EDE14196E1AC0C6
:10194000D9FF1BC0DAFFDECF0BF01C940BBC1C844C
:101950001C960BBE1C86DFCF0CF0DCCF1FF0DD50D9
:101960001F38070B1F6E0B38030B0A625ED0125034
:1019700014625BD01350156258D0030E0C1455E05E
:101980001C9216B91C82020EDFBE1C1A1F50040ADC
:1019900003E0060E1F6210D01CB207D002EE7DF0ED
:1019A0000F50E9261050EF1206D002EE7DF00F50D6
:1019B000E926101CEF161C82020E0A620FD00AC024
:1019C00020F0299029921CB229820EC021F00FC06C
:1019D00022F01050CCEC13F0010127D01CB415D02C
:1019E0001CA613D00EA011D00AC020F029901CB460
:1019F000298029821CB229920EC021F00FC022F04A
:101A00001050CCEC13F0010110D00AC020F0299046
:101A10001CB4298029921CB229820EC021F00FC06B
:101A200022F01050CCEC13F00101030ED926000E69
:101A3000DA22DFCF0DF0D8900C32D8900C32030EA2
:101A40000C14D8B480D01C9216B91C82030E0C144E
:101A5000010A05E0030A06E0010A06E074D01CB2A0
:101A600003D071D01CB26FD00DAE47D012501662A9
:101A70006AD01350176267D0020E0DBC1C1A1F509B
:101A8000040A03E0060E1F6210D01CB207D002EE5B
:101A90007DF00F50E9261050EF1206D002EE7DF0D7
:101AA0000F50E926101CEF161C821CB415D01CA682
:101AB00013D00EA011D00AC020F029901CB42980A8
:101AC00029821CB229920EC021F00FC022F01050C2
:101AD000CCEC13F0010137D00AC020F029901CB4DF
:101AE000298029921CB229820EC021F00FC022F059
:101AF0001050CCEC13F0010126D01250146203D028
:101B00001350151808E0125018621DD013501962B6
:101B10001AD01EAE18D002EE6DF00F50E926EFCFAE
:101B200011F01CA203D01050111202D0101C11167B
:101B300002EE6DF00F50E92611C0EFFF03EE60F0EA
:101B4000E9261050EF12020ED926000EDA22DFCF5E
:101B50000DF0D8900C32D8900C32030E0C14D8B47F
:101B600080D01C9216B91C82030E0C14010A05E0E9
:101B7000030A06E0010A06E074D01CB203D071D05B
:101B80001CB26FD00DAE47D0125018626AD01350FD
:101B9000196267D0020E0DBC1C1A1F50040A03E024
:101BA000060E1F6210D01CB207D002EE7DF00F505F
:101BB000E9261050EF1206D002EE7DF00F50E92614
:101BC000101CEF161C821CB415D01CA613D00EA03E
:101BD00011D00AC020F029901CB4298029821CB29F
:101BE00029920EC021F00FC022F01050CCEC13F05F
:101BF000010137D00AC020F029901CB42980299215
:101C00001CB229820EC021F00FC022F01050CCEC83
:101C100013F0010126D01250146203D0135015188E
:101C200008E0125016621DD0135017621AD01DAE74
:101C300018D002EE75F00F50E926EFCF11F01CA27C
:101C400003D01050111202D0101C111602EE75F0C4
:101C50000F50E92611C0EFFF03EE68F0E92610509F
:101C6000EF12D89010361DD60F2A15D6125012003A
:101C700001010751E96E050E0825EA6E0B0EEF6EA5
:101C800088D90751E96E050E0825EA6EED0EEF6E54
:101C900080D90751E96E050E0825EA6E0B0EEF6E2E
:101CA00078D90751E96E050E0825EA6E7F0EEF6EB2
:101CB00070D90751E96E050E0825EA6E310EEF6EF8
:101CC00068D97F38E8441F0B7F6E7F3A7F42F80E59
:101CD0007F16030E7F147F12D8907F36700E7F1A06
:101CE0007F807F9ED8907F32D8907F320751E96EF7
:101CF000050E0825EA6E010EEF6E4BD90751E96E0D
:101D0000050E0825EA6E7FCFEFFF43D90751E96E34
:101D1000050E0825EA6E7FCFEFFF3BD90751E96E2C
:101D2000050E0825EA6E7FCFEFFF33D90751E96E24
:101D3000050E0825EA6EEF6A2CD90751E96E050EEB
:101D40000825EA6EEF6A25D90551075D7F6E0651B9
:101D500008597F6E7FAE02D0020E7F267FBE06D06E
:101D6000E10E7F5C010E7F58D8B02D98050E020160
:101D7000036F3E6A12007F6E7F68010113AD1AD0B7
:101D80007F38E8461F0B1F0B7F6E7F38E8461F0B1E
:101D90001F0B7F6E070E7F167F167F507F6228D045
:101DA0007F507F6225D07F6A7F507F6221D0010EF5
:101DB0007F6E1ED07F38030B7F6E7F38E840E8428D
:101DC0003F0B030B7F6E7F507F6212D00F0E7F168A
:101DD0007F147F6E7F507F6E7F507F6209D07F506F
:101DE0007F6206D0000E7FB8010E7F6E7F507F1A93
:101DF0007F501200032B04EE00F00351E926EF5050
:101E00000B0A03E00A680B68FF0C032B04EE00F0DA
:101E10000351E926EF507F0A03E00A680B68FF0CC4
:101E2000032B04EE00F00351E926EF38070B030AF9
:101E300003E00A680B68FF0C032B04EE00F003516B
:101E4000E926070EEF14010A03E00A680B68FF0C8D
:101E5000032B04EE00F00351E926EFCF0AF00AACA1
:101E600003D00A680B68FF0CD8900A36D8900A365F
:101E7000032B04EE00F00351E926EFCF0BF0700EB8
:101E80000B1AD8900B32030E0B140A120B3A0B46A6
:101E90001F0E0B16032B04EE00F00351E926EFCFC3
:101EA0000CF00C3A0C42F80E0C160C500B120A50A7
:101EB000120004EE00F00351E926EFCF0CF0032BE3
:101EC00004EE00F00351E926D890EF340A6E032B9C
:101ED00004EE00F00351E926EFCF0DF004EE00F020
:101EE000E9263F0EEF140B6E0E900DBC0E80030E14
:101EF0000C14020A05E0030A0DE0010A1EE032D0CC
:101F00000EB003D00A680B68FF0C0A900DBA0A8065
:101F10000B8E28D00EB00BD00DBA02D00DA804D075
:101F20000DAA05D00DA803D00A680B68FF0CD89045
:101F30000B320A320B960B8C15D00EA003D00A6818
:101F40000B68FF0CD8900B320A320BB60AD00AC0CD
:101F50000FF00BC010F007012ED80A680B680101C2
:101F6000FF0C0B960A5012003E50D8A4800C03C2FE
:101F700005F213878B900101800C3F500101D8A41A
:101F8000800C040E0201086F010113898B9401017A
:101F9000800C072B000E0823076705D0020E08638C
:101FA00002D0076B086B120009A503D00101106B6A
:101FB000128D01011200070E1014166E0F50156ECF
:101FC000F80E155C030E1658D8A0D2D0FC0E155C86
:101FD000030E1658D8B0CCD0030E0F14146E10B8E0
:101FE0001484116A080E1160BED01268010E136EBF
:101FF0001352D8B4B6D0122A1150400DF3CFD9FFE6
:10200000F4CFDAFF100ED926070EDA22080E1202DC
:10201000F350D926000EDA22DECF17F0DF38030B9B
:10202000196E0F0EDE14186E18BC98D0030E1C6EBD
:10203000D890183217321C2EFBD7186A070E1716C5
:10204000DECF1AF01B901ABC1B80030E1A141BE083
:102050001750146218D009A70AD01BA008D0195233
:1020600006E003EE40F01150E9261350EF1209A9E3
:102070000AD01BB008D0196606D003EE40F011500C
:10208000E9261350EF12DE50DECF17F0DF380F0BCA
:10209000196E1B9019B61B80030E19160F0EDE1455
:1020A000186E030E1C6ED890183217321C2EFBD7F8
:1020B000186A070E17160C0E1A141BE0175014623C
:1020C00018D009A70AD01BB008D0195206E003EEB9
:1020D00060F01150E9261350EF1209A90AD01BA095
:1020E00008D0196606D003EE60F01150E9261350AF
:1020F000EF12DECF17F0DF380F0B196E1B9019B6F9
:102100001B80030E19160F0EDF14186E030E1C6EC3
:10211000D890183217321C2EFBD7186A070E1716E4
:10212000300E1A141BE01750146218D009A70AD0F9
:102130001BB008D0195206E003EE68F01150E926F2
:102140001350EF1209A90AD01BA008D0196606D0B7
:1021500003EE68F01150E9261350EF12D8901336B1
:1021600047D7112A3FD7180E091502E00101128B3B
:10217000070112001B6E030EEA6E1AC0E9FF1B4630
:102180001B461B44060FF924D8B0FA2AF96EEF6AF1
:10219000000E00003BD00A0EEF6E000E37D0140E7A
:1021A000EF6E000E33D0230EEF6E000E2FD0320EE6
:1021B000EF6E000E2BD0410EEF6E000E27D0500EAA
:1021C000EF6E000E23D0640EEF6E000E1FD07D0E5A
:1021D000EF6E000E1BD0960EEF6E000E17D0C80EDD
:1021E000EF6E000E13D02C0EEF6E010E0FD0900E7E
:1021F000EF6E010E0BD0F40EEF6E010E07D0580EED
:10220000EF6E020E03D0200EEF6E030EEC6E120086
:102210001B6E030EEA6E1AC0E9FF1B461B46F950FF
:102220001B44F926E80EEF6E030E3BD0DC0EEF6E7A
:10223000050E37D0D00EEF6E070E33D0B80EEF6E0E
:102240000B0E2FD0A00EEF6E0F0E2BD0880EEF6E60
:10225000130E27D0700EEF6E170E23D0280EEF6EE0
:10226000230E1FD0E00EEF6E2E0E1BD0500EEF6E21
:10227000460E17D0C00EEF6E5D0E13D0300EEF6E0F
:10228000750E0FD0A00EEF6E8C0E0BD0100EEF6EF1
:10229000A40E07D0800EEF6EBB0E03D0600EEF6E63
:1022A000EA0EEC6E12001B6E030EEA6E1AC0E9FF16
:1022B0001B461B461B44060FF924D8B0FA2AF96EB8
:1022C000050EEF6E000E3BD00A0EEF6E000E37D0FB
:1022D000140EEF6E000E33D0230EEF6E000E2FD0D3
:1022E000320EEF6E000E2BD0410EEF6E000E27D097
:1022F000500EEF6E000E23D0640EEF6E000E1FD056
:102300007D0EEF6E000E1BD0960EEF6E000E17D0F6
:10231000C80EEF6E000E13D02C0EEF6E010E0FD014
:10232000900EEF6E010E0BD0F40EEF6E010E07D083
:10233000580EEF6E020E03D0200EEF6E030EEC6E01
:10234000120013B541D0070109A13ED0F29E100E34
:102350000A6E020E0B6E0C6A080E02010C6010D0A1
:102360000AC012F00BC013F003EE20F00C50E92667
:10237000EF501FEC1CF00A2A000E0B220C2AECD79F
:10238000002B000E012302230A0E0A6E0B6A0AC0FC
:1023900012F00BC013F000511FEC1CF00A2A000EC3
:1023A0000B220AC012F00BC013F001511FEC1CF0FD
:1023B0000A2A000E0B220AC012F00BC013F00251C1
:1023C0001FEC1CF0010113852B0EC26E0201C2B27C
:1023D000FED7030EC4140101186FC3CF17F11D0EF1
:1023E000175D010E185909E28B90640E166E08D81D
:1023F0008B80640E166E04D8E7D7D190FF001200D0
:10240000176A1650176009D0A192B10EB36EB18051
:10241000A1A2FED7B190172AF4D71200F95039447F
:10242000F92602D006D02FD0566A080E566041D148
:10243000010C03EE40F05650E926EF50D8B437D1E6
:1024400003EE00F05650E926EF50D8B430D154686E
:10245000010E556E5552D8B42AD1542A03EE40F0DD
:102460005650E926EFCF57F003EE00F0E926EF5083
:10247000571655505714D8B417D103EE40F05650A4
:10248000E926551CEF162DA8020C5650400DF3CF2F
:10249000D9FFF4CFDAFF100ED926070EDA22080E84
:1024A0005402F350D926000EDA22DECF5AF05B6ACE
:1024B000DFCF5BF0DECF0AF0DFCF0BF0DECF0CF02A
:1024C000DECF0DF003EE20F05650E9265550EF1404
:1024D0005B88D8B45B985AC058F05BC059F00A3892
:1024E000030B03E112AB64D0DFD00D38070B60E1C2
:1024F00012BB5ED003EE10F05650E9265550EF1493
:1025000016E003EE10F05650E926551CEF1603EEC8
:1025100048F05650E9265550EF14D880D8B4D890DA
:1025200003E25BB8C1D044D05BB842D0BDD003EE6B
:1025300058F05650E9265550EF1424E103EE48F0C8
:102540005650E926551CEF165BA813D003EE48F051
:102550005650E9265550EF12030E0C14030A28E0DA
:102560000DC00FF054C010F056C011F05550A4D853
:102570009BD00DC00FF054C010F056C011F0555054
:102580009BD892D003EE48F05650E9265550EF14F0
:10259000D880D8B4D89003E25BB803D009D05BB838
:1025A00007D003EE58F05650E926551CEF167CD0A4
:1025B000030E0C14010A07E0030A08E0010A08E010
:1025C000030A38E005D05BB803D034D05BB832D012
:1025D00003EE38F05650E926EFCF0EF05BAC03D097
:1025E00055500E1A08D05BB802D0551C0E165BA8C9
:1025F00002D055500E1255500E145B88D8B45B981B
:1026000003EE38F05650E9260EC0EFFF000E5BB81F
:10261000010E0BAE04D0000A5B98D8B45B880AC0E8
:102620000FF016905AC010F05BC011F05450A8EC97
:102630000BF0010158C05AF059C05BF012BB34D006
:10264000D8900C32D8900C32030E0C14010A07E01B
:10265000030A08E0010A08E0030A0CE005D05BB8B1
:1026600003D008D05BB806D003EE60F05650E926E0
:102670005550EF12D8900C32D8900C32030E0C1437
:10268000010A07E0030A08E0010A08E0030A0CE077
:1026900005D05BB803D008D05BB806D003EE68F075
:1026A0005650E9265550EF12D8905536D3D6562AB3
:1026B000BCD6000C0101800C126E0F0E0F14136EAD
:1026C0000F38070B146E020A02E014662AD0080EB7
:1026D0001102F3501024156E135207E0D8901534F0
:1026E000700F1A6E135046DD16D0020E146209D018
:1026F00003EE70F0D8901534E9260A0EEE6EEF6AFC
:102700000AD0146608D003EE70F0D8901534E9268C
:10271000010EEE6EEF6A03EE58F01150E9261250EA
:10272000EF1212000A500B14FF0AD8B4120027EE61
:1027300010F0116A080E11602ED00F6A010E106E93
:10274000105227E0DECF0CF0DFCF0DF00DBE19D018
:10275000070E0D16DECF0EF0129016B912800E384D
:10276000030B0FE10A500C620CD00B500D6209D024
:102770002C9012B02C80300E11242A6E10509AEC3E
:1027800018F0060ED926000EDA220F2AD89010363D
:10279000D7D7112ACFD71200236E020129B013D048
:1027A0002C9029B22C80200E22242A6E23509AECE1
:1027B00018F003EE40F02250E9262350EF12050EE8
:1027C000036F3E6AD4D02066D2D021B007D003EE8A
:1027D00058F02250E926231CEF1608D003EE58F0DB
:1027E0002250E926D8902330FF0AEF1621B027D0D7
:1027F0002C8029B22C90200E22242A6E23509AEC91
:1028000018F02C8029B22C90180E22242A6E235006
:102810009AEC18F02C9029B22C80200E22242A6EDB
:10282000D89023349AEC18F02C9029B22C80180EF2
:1028300022242A6ED89023349AEC18F098D029B22A
:102840001FD02C90200E22242A6E23509AEC18F0D0
:102850002C90180E22242A6E23509AEC18F02C90FB
:10286000200E22242A6ED89023309AEC18F02C9057
:10287000180E22242A6ED89023309AEC18F077D0C4
:10288000D9CF27F0DACF28F02250400DF3CFD9FF6F
:10289000F4CFDAFF130ED926070EDA22080E210232
:1028A000F350D926000EDA220F0EDF14256E2550C4
:1028B00006E0050A04E00F0A02E0050A27E12C9071
:1028C00025B22C80200E22242A6E23509AEC18F078
:1028D0002C9025B22C80180E22242A6E23509AECBC
:1028E00018F02C9025B02C80200E22242A6ED8902F
:1028F00023309AEC18F02C9025B02C80180E22244E
:102900002A6ED89023309AEC18F02DD02C80200E0F
:1029100022242A6E23509AEC18F02C80200E2224B8
:102920002A6ED89023309AEC18F0080ED95E000E6B
:10293000DA5A5F0EDF1417E0060E2114266E080E19
:102940002202F3502624246E03EE70F0D890243433
:10295000E926010EEE6EEF6A03EE58F02250E926EA
:10296000D8902330EF1227C0D9FF28C0DAFF120019
:102970000101F9503844F92602D01BD033D05D6AEA
:102980000001080E5D60C8D003EE40F05D50E926FE
:10299000EFCF5FF003EE00F0E926EF1C5F14D8B430
:1029A000B9D05C68010E5E6E5E52D8B4B3D05C2ABA
:1029B000010C03EE40F05D50E926EFCF5FF003EE2F
:1029C00000F0E926EF1C5F165E505F140001D8B4DA
:1029D0009ED003EE40F05D50E9265E1CEF1601012B
:1029E00012AB3AD000012DA8020C5D50400DF3CF80
:1029F000D9FFF4CFDAFF110ED926070EDA22080E1E
:102A00005C02F350D926000EDA22DDCF0BF00BBCAE
:102A10007ED00B38030B7BE1DECF0CF00D6ADECFEE
:102A20000DF003EE20F05D50E9265E50EF140D88A6
:102A3000D8B40D98DFAE04D0000A0D98D8B40D8834
:102A4000100E0F6E16900CC010F00DC011F05C50FF
:102A5000A8EC0BF000015BD05D50400DF3CFD9FF27
:102A6000F4CFDAFF110ED926070EDA22080E5C0227
:102A7000F350D926000EDA22DECF60F0DECF61F00F
:102A8000DECF62F00F0E00016215636F6239070B33
:102A9000626F030E61150CE062C010F063C011F0AC
:102AA00060C012F05CC013F05DC014F05E5045D9F8
:102AB000DCCF0AF0D8906133D8906133030E6115F2
:102AC0000EE00AAE0CD062C010F063C011F060C01E
:102AD00012F05CC013F05DC014F05E502ED9DE50D1
:102AE000DCCF0AF0D8906133D8906133030E6115C2
:102AF0000EE00AAE0CD062C010F063C011F060C0EE
:102B000012F05CC013F05DC014F05E5016D9D8907E
:102B10005E364AD75D2A35D7000CF9503C44F92679
:102B200002D012D01FD0666B080E66617DD003EE16
:102B300060F06651E926EF5075E06469010E656F3B
:102B4000655370E0642B010C03EE40F06651E926FA
:102B50006551EF1464E103EE60F06651E9266551BA
:102B6000EF145DE02DA8020C03EE60F06651E9263B
:102B7000651DEF166651400DF3CFD9FFF4CFDAFF94
:102B8000100ED926070EDA22080E6403F350D92658
:102B9000000EDA22DCCF0AF0030ED926000EDA226C
:102BA000DECF0BF00C6A3F0EDF140C6EDFCF0DF0A2
:102BB00002EE6DF06651E9266551EF140C88D8B429
:102BC0000C980E900ABE0E8003EE00F06651E926C6
:102BD0006551EF140EE00EB00CD00A38030B09E17A
:102BE00003EE30F06651E9266551EF140C88D8B435
:102BF0000C98010112AB07D00D38030B0F6E0F6656
:102C000002D0100E0D6E0DC00FF016800BC010F02C
:102C10000CC011F000016451A8EC0BF00001D89039
:102C200065378ED7662B80D7800CF9503D44F92646
:102C300002D012D01FD0686B080E68617DD003EE01
:102C400068F06851E926EF5075E06969010E676F19
:102C5000675370E0692B010C03EE40F06851E926E0
:102C60006751EF1464E103EE68F06851E92667519B
:102C7000EF145DE02DA8020C03EE68F06851E92620
:102C8000671DEF166851400DF3CFD9FFF4CFDAFF7F
:102C9000100ED926070EDA22080E6903F350D92642
:102CA000000EDA22DCCF0AF0050ED926000EDA2259
:102CB000DECF0BF00C6A3F0EDF140C6EDFCF0DF091
:102CC00002EE75F06851E9266751EF140C88D8B40C
:102CD0000C980E900ABE0E8003EE00F06851E926B3
:102CE0006751EF140EE00EB00CD00A38030B09E167
:102CF00003EE30F06851E9266751EF140C88D8B420
:102D00000C98010112AB07D00D38030B0F6E0F6644
:102D100002D0100E0D6E0DC00FF016800BC010F01B
:102D20000CC011F000016951A8EC0BF00001D89023
:102D300067378ED7682B80D7800C156E03EE20F096
:102D40001450E9261550EF14D8B48DD0080E140293
:102D5000F3501324166E105203E0020E106208D0D6
:102D6000D8901634700F1A6E1150BAEC10F01AD0B9
:102D7000104C03D0030E106208D0D8901634700F98
:102D80001A6E115008EC11F00DD01050040A03E037
:102D9000060E106207D0D8901634700F1A6E1150BC
:102DA00053EC11F003EE70F0D8901634E926EECF14
:102DB00018F0EECF19F01050020A0BE0010A14E0EF
:102DC000050A12E0060A2DE0010A36E0050A34E0A1
:102DD00048D01850191008E103EE18F01450E926F5
:102DE0001550EF12D890120003EE58F01450E92657
:102DF0001550EF1436E103EE18F01450E926155083
:102E0000EF1A03EE70F0D8901634E92618C0EEFFE2
:102E100019C0EEFF03EE58F01450E9261550EF12DA
:102E200020D01850191008E103EE18F01450E926CC
:102E30001550EF12D890120003EE18F01450E92646
:102E40001550EF1203EE70F0D8901634E92618C032
:102E5000EEFF19C0EEFF03EE58F01450E9261550AE
:102E6000EF12D88012001050020A0BE0010A09E0AC
:102E7000050A07E0060A0BE0010A09E0050A07E077
:102E80000CD003EE58F01450E926151CEF1603EE93
:102E900018F01450E926151CEF16D8901200F950BE
:102EA0003B44F92601D005D06A6B080E6A61B6D0A2
:102EB000010C03EE58F06A51E926EF50D8B4ACD0BB
:102EC0000B68010E0A6E0A52D8B4A6D00B2A03EE84
:102ED00058F06A51E9260A50EF14D8B499D06A51D3
:102EE000400DF3CFD9FFF4CFDAFF100ED926070E2D
:102EF000DA22080E0B02F350D926000EDA22DCCFBC
:102F00000CF0DCCF0EF0DCCF0DF00D38070B0F6EA0
:102F100003EE70F0080E6A03F3500B24D890E834E7
:102F2000E926EE06000EEF5A03EE70F0080E6A0373
:102F3000F3500B24D890E834E926EE50EF1068E106
:102F400003EE00F06A51E926EF1C0A144FE00CACC6
:102F500019D0080ED926000EDA220D38F00B0D6EAE
:102F60000F0EDF140D26080ED95E000EDA5A0FC0C0
:102F700010F00DC011F00BC012F06AC013F00A502F
:102F80004ED846D00F50020A06E00F50030A03E065
:102F9000060E0F6213D003EE58F06A51E9260A1CA0
:102FA000EF160FC010F00F0E0D14116E126A0BC049
:102FB00013F06AC014F00A50C0DE14D00F5205E0BE
:102FC0000F4C03D0040E0F620DD003EE58F06A517F
:102FD000E9260A1CEF1603EE18F06A51E9260A1CCE
:102FE000EF1616D0010112AB13D012D003EE58F039
:102FF0006A51E9260A1CEF1603EE10F06A51E92621
:103000000A50EF1203EE40F06A51E9260A50EF121F
:10301000D8900A36000157D76A2B47D7800C146E18
:1030200003EE18F01350E926196AEFCF18F012508A
:1030300005E01A6ED89018321A2EFCD7196A030EC2
:1030400018161114186212D02C9011B42C80180E7E
:1030500013242A6E14506ED82C9011B62C80180EA2
:1030600013242A6ED890143465D811D02C9011B046
:103070002C80180E13242A6E14505CD82C9011B298
:103080002C80180E13242A6ED890143453D811387B
:103090000F0B116E080E1302F3501224156E03EE7F
:1030A00058F01350E926141CEF161050020A05E0E0
:1030B000010A1DE0050A1BE033D0D8901534700FCB
:1030C0001A6E1150BAEC10F003EE70F0D89015346F
:1030D000E926EECF16F0EECF17F01650171020E0CD
:1030E00003EE58F01350E9261450EF1219D0D8907F
:1030F0001534700F1A6E115008EC11F003EE70F0D9
:10310000D8901534E926EECF16F0EECF17F0165012
:10311000171006E003EE58F01350E9261450EF1292
:1031200003EE70F0D8901534E92616C0EEFF17C0F4
:10313000EEFF12002B6E030EEA6E2AC0E9FFD89054
:103140002B50EF14D8A4D8802CA003D02B50EF1212
:1031500002D02B1CEF1612003A50D8A4800C6B2B17
:10316000080E6B616B6B03EE18F06B51E926EFCF25
:103170000AF003EE50F0E926EF500A1A03EE00F0D1
:103180006B51E926EF1C0A1603EE00F06B51E9269D
:10319000EF4812D001EE27F06B51E9260AC0EFFF8D
:1031A0006BB103D0150E6C6F02D0140E6C6F6BC038
:1031B0000CF06C517FD800016BB103D0130E6C6F13
:1031C00002D0120E6C6F03EE00F06B51E926EF5047
:1031D00034E06BC00BF06C5101019DD803EE00F0A0
:1031E00000016B51E926EF1C0A6E03EE08F06B51EB
:1031F000E9260A50EF1601EE27F06B51E926EFCFD2
:103200000AF003EE00F0E926EF500A1603EE08F08C
:103210006B51E9260A50EF1203EE50F06B51E9268C
:10322000EFCF0AF003EE00F0E926EF500A1603EEA6
:1032300008F06B51E9260A50EF1A000C4050D8A450
:10324000800C0A6A080E0A6034D003EE00F00A50BF
:10325000E926EFCF0BF00AB015D001EE27F0E926F2
:103260000BC0EFFF0AC00CF0010E24D801EE27F0CE
:103270000A50E926EF6A0AC00CF0150E00011AD8B0
:10328000000115D001EE27F00A50E9260BC0EFFF30
:103290000AC00CF0000E0ED801EE27F00A50E92605
:1032A000EF6A0AC00CF0140E000104D800010A2ACB
:1032B000C9D7800C0D6E0101F00E116E12681F0E41
:1032C000C5140E6E070EC7140F6E0E66FED70F667E
:1032D000FCD7060E0C14226F228D0DC023F1010EB7
:1032E000216F01EE27F00C50E926EFCF24F10CB04E
:1032F00042D89E969D86C58021530CE01106000E93
:10330000125A1150121002E0213DF6D70C28136E0C
:1033100060D8D2D712000C6EF00E0F6E10681F0E20
:10332000C5140D6E070EC7140E6E0D66FED70E6621
:10333000FCD7060E0B14226F228D0CC023F1020E57
:10334000216F9E969D86C58021530CE00F06000ECE
:10335000105A0F50101002E0213DF6D70B28136EC3
:1033600038D8DAD70BB007D801EE27F00B50E92692
:1033700024C1EFFF120024C114F014C013F0F00EAA
:103380001314E83A0F0B136E0F0E1414E83AF00BF7
:10339000146E131213C014F0CC0E1316D8901332FF
:1033A000D8901332330E1416D8901436D8901436A1
:1033B0001450131213C014F0AA0E1316D89013321F
:1033C000550E1416D89014361450131213C024F14D
:1033D0001200020E156E8B80146A135014600CD00C
:1033E0008B900A0E166E00EC12F08B80280E166E73
:1033F00000EC12F0142AF1D7C80E166E00EC12F091
:10340000152EE9D79E969D96148BC590C66A280EF8
:10341000C66E1200032B032B04EE00F00351E926C5
:103420007C0EEF625CD0032B04EE00F00351E92622
:10343000EFCF0CF0032B032B04EE00F00351E92631
:10344000EFCF0BF0032B04EE00F00351E926D890E8
:10345000EF340A6E0B340B320A320A5002016B63EE
:1034600004D00B506C6301D00BD0010113AF07D017
:103470000F0E0A6204D0270E0B6201D001D0120099
:103480000101032B032BFC0E0C14200A0BE0080A8D
:1034900009E0040A11E04C0A19E0080A17E00C0AD6
:1034A0001AE01DD00CC00DF00AC00EF00BC00FF0DA
:1034B00017D8010E74D913D00CC00DF00AC00EF04D
:1034C0000BC00FF00DD8010E6AD909D0DFD8400E1D
:1034D000010165D904D0DAD8400E010160D912008B
:1034E00012EE2BF00E0EE66EE70EE66E0E0EE66E98
:1034F0007C0EE66E0DC0E6FFE66AD8900E360F36FB
:10350000D8900E320FC0E6FF0EC0E6FFE66A166ADC
:1035100004EE00F00351E926EFCF14F014C013F0CD
:1035200013380F0B136E032B04EE00F00351E92642
:10353000EFCF15F015C012F0129E14B0128E179036
:10354000125013100AE1040E126E136AE96E070E90
:103550001324EA6EEFCF16F01780135003E1050E27
:10356000126412D0135010E1090E12600DD0060E35
:10357000125E000E135A1250E96E070E1324EA6E03
:10358000EFCF16F017806DD0100E126202D01352DA
:1035900005E0110E12620FD013660DD00C0E125EF4
:1035A000000E135A1250E96E070E1324EA6EEFCF85
:1035B00016F0178056D01B0E126202D0135205E08F
:1035C0001C0E12620FD013660DD0150E125E000E87
:1035D000135A1250E96E070E1324EA6EEFCF16F05D
:1035E00017803FD06F0E12620FD013660DD0660E9B
:1035F000125E000E135A1250E96E070E1324EA6E83
:10360000EFCF16F017802DD0135003E16F0E126428
:1036100012D0135010E1730E12600DD0660E125EC0
:10362000000E135A1250E96E070E1324EA6EEFCF04
:1036300016F0178016D0135002E112AE12D0810E90
:10364000125C020E13580DE2800E125E000E135A29
:10365000100E1224E96E070E1320EA6EEFCF16F05B
:103660001780149216BE148214C0E6FF15C0E6FF40
:103670007F0E1614E66EE66AE66A17A005D0050E00
:103680000201036F3E6A010113831200119004EEE0
:1036900000F00351E926EFCF10F0032B04EE00F009
:1036A0000351E926EFCF0FF00F9E10B00F8E032BC2
:1036B00004EE00F00351E926EFCF0DF00D9E10B29D
:1036C0000D8E10380F0B106E100E0F6202D01052BC
:1036D00005E0110E0F620ED010660CD00C0E0F5EBE
:1036E000000E105A0F50E96E070E1024EA6E0DC03E
:1036F000EFFF45D01B0E0F6202D0105205E01C0EEA
:103700000F620ED010660CD0150E0F5E000E105A10
:103710000F50E96E070E1024EA6E0DC0EFFF2FD098
:103720006F0E0F6210D010660ED0660E0F5E000E88
:10373000105A0F50E96E070E1024EA6E800E0D101D
:10374000EF6E11801CD0105002E10FAE17D0800E2A
:103750000F5C020E105812E2800E0F5E000E105A1F
:10376000100E0F24E96E070E1020EA6E0DC0EFFF59
:10377000100E0F26000E1022118001D012000FC073
:1037800012F010C013F00D505AD811A003D019D95F
:10379000406A88D9050E0201036F3E6A12000D6E61
:1037A0000751E96E050E0825EA6E040EEF6EC9ECAE
:1037B0000FF00751E96E050E0825EA6EB40EEF6EA4
:1037C000C9EC0FF00751E96E050E0825EA6E6F0E81
:1037D000EF6EC9EC0FF00751E96E050E0825EA6E91
:1037E0000DC0EFFFC9EC0FF00551075D0E6E0651DD
:1037F00008590F6E0FAE02D0020E0F260FBE06D074
:10380000E10E0E5C010E0F58D8B02D981200032B5C
:1038100004EE00F00351E9266F0EEF6204D013A30B
:1038200002D01393366A1200A6B2FED715C0A9FFC4
:1038300016C0AAFFA69EA69CA680A8501200146ED1
:1038400012C015F013C016F0EFDF14181CE0A6B27A
:10385000FED714C0A8FF12C0A9FF13C0AAFFA69EDE
:10386000A69CA684F29E550EA76EAA0EA76EA682EF
:10387000F28EA69412C015F013C016F0D5DF1418FE
:1038800002E0D8901200D88012007FCFF6FF7FCFE1
:10389000F7FFF86AA68EA69C0800F5501200F00EFD
:1038A000D36EC00E9B6E100E386F020E396F040E71
:1038B0003A6F110EC26EC16ABE0EC06E806A200ED3
:1038C000926E816AF30E936E616A050E826EFA0E35
:1038D000946E270EC86E280EC66EC56ACB6AC76A7C
:1038E000200EAC6E900EAB6EB86A3B0EAF6EF26AF5
:1038F000F16AF06A9D6AA06A9F6AA26AD59ED66A3A
:10390000CD6ABA6A300EB16E2B0EC26E0101C2B220
:10391000FED7030EC414186FC3CF17F1180E175D2E
:10392000010E18590BE28B90640E166E00EC12F02B
:103930008B80640E166E00EC12F0E6D70FEE37F0B7
:10394000ED6AEA50FDE1E950FBE1EF6A0D01928377
:1039500082A202D0D8901200D880120007EE00F0A8
:103960000A6A0B6A0AC015F00BC016F05DDFEE6E36
:103970000A2A000E0B221C0E0A5C020E0B58F2E300
:103980000AC700F20BC701F20CC702F23F0E070193
:10399000041502016C6F05C76BF201011481A68E3C
:1039A000A69CF66AF76A200EF86E0EEE40F0080E3E
:1039B000106E0900F5CFEEFF102EFBD745CE48FE66
:1039C000120027EE12F0156A080E156027D0010EBE
:1039D000146E03EE50F01550E926EF6A03EE00F086
:1039E000E926EF6ADFAC07D003EE00F01550E926B8
:1039F0001450EF1209D0DCAE06D003EE50F0155093
:103A0000E9261450EF12DD50D8901436080ED9264E
:103A1000000EDA221466E6D7152AD6D7120009A1BD
:103A200040D027EE11F00B6A080E0B603AD0010E61
:103A30000D6E0C6ADFCF0EF0020ED926000EDA22D0
:103A4000DFCF0FF00F38070B0F6E0EBC04D0040A47
:103A500002E00D500C12D8900D36060ED926000E3D
:103A6000DA220D66E7D7100E0B24E96E090EEA6A1A
:103A7000EA22EFCF0AF003EE20F00B50E9260C50BB
:103A80000A14EF6E03EE00F00B50E926EF1C0A6EED
:103A900003EE40F00B50E9260C500A14EF6E0B2A8F
:103AA000C3D712000101016B126A100E12600CD014
:103AB000080E1202F350100FD96E070EDA6ADA22DE
:103AC000DF500127122AF1D7040E02016B03F350D5
:103AD000010101273F0E011701C106F712000A6A12
:103AE00001510A600BD0A192B368B26AB180A1A261
:103AF000FED7B19012B502D00A2AF2D71200020EF8
:103B00007F6EA68EA69CA684A68EF66AF76AF86AD1
:103B1000A688550EA76EAA0EA76EA682A6980A00C2
:103B20000EEE00F0400E7F6EEECFF5FF0F007F0629
:103B30007F50FAE1550EA76EAA0EA76EA682A69434
:103B4000F66A0EEE00F07F80400E7F6E0900F550A1
:103B5000EE1802E07F9003D07F067F50F7E17FA050
:103B600002D0D88012007F067F50CDE1D89012009D
:0200000400F00A
:1000000011571800270F00E0009F000000000000BB
:100010000020430000000000012043000000000019
:100020000220430000000000032043000000000005
:1000300004204300000000000520430000000000F1
:1000400006204300000000000720430000000000DD
:1000500008204300000000000920430000000000C9
:100060000A204300000000000B20430000000000B5
:100070000C204300000000000D20430000000000A1
:100080000E204300000000000F204300000000008D
:100090001020430000000000112043000000000079
:1000A0001220430000000000132043000000000065
:1000B0001420430000000000152043000000000051
:1000C000162043000000000017204300000000003D
:1000D0001820430000000000192043000000000029
:1000E0001A204300000000001B2043000000000015
:1000F0001C204300000000001D2043000000000001
:100100001E204300000000001F20430000000000EC
:1001100020204300000000002120430000000000D8
:1001200022204300000000002320430000000000C4
:1001300024204300000000002520430000000000B0
:10014000262043000000000027204300000000009C
:100150002820430000000000292043000000000088
:100160002A204300000000002B2043000000000074
:100170002C204300000000002D2043000000000060
:100180002E204300000000002F204300000000004C
:100190003020430000000000312043000000000038
:1001A0003220430000000000332043000000000024
:1001B0003420430000000000352043000000000010
:1001C00036204300000000003720430000000000FC
:1001D00038204300000000003920430000000000E8
:1001E0003A204300000000003B20430000000000D4
:1001F0003C204300000000003D20430000000000C0
:100200003E204300000000003F20430000000000AB
:0C021000000000000000000000000000E2
:020000040000FA
:0400000000EF02F01B
:020000040030CA
:0E000000FF280008FF8181FF0FC00FE00F40B6
:00000001FF
